S113C7007EC7217EC7037EC7477EC7857EC7957EC9
S113C710C71F0C00000000C810C810000000003B38
S113C720121A10BECC3110EF027DCC3426118ECCFF
S113C730FC7CCC346D842707BFCC3110EE023B8ED9
S113C740CCF87FCC3420F11A107DC71B2729BEC733
S113C75019A6843402EC018ECAC0ED88403502A7C4
S113C760036F848601A7026F88226F883B7DC71EF2
S113C7702729113F1220F61CEFAD9FD3ED7FCCFC8F
S113C780113F1220F41A107DCC302705113F1220DE
S113C790F47CCC30397FCC301CEF397DC71D262783
S113C7A08ECAC0BDD406261F7DC71C270F7FC71C99
S113C7B0810A270F3402860A8D3C3502810D260337
S113C7C0B7C71C8D3120D4860D8D2B860A8D27B6D4
S113C7D0C7128D227FC71DBEC7196D0327056A03C3
S113C7E07EC74730048CC84026038EC810BFC719C3
S113C7F07AC71B7EC747BDCCD82B05113F1220F644
S106C8007ECCE403
S113C840FF000000535441525455500054585400B2
S113CA002006BDCAAC39C0A08639B7D3FDBECC2B35
S113CA10308900A1BFCA06AD9FD3F1BED3FBBFCD01
S113CA200ABFCD0DBED3F9BFCD10BFCD13BED3F712
S113CA30BFCD4F8E00A0C6B9A684E78412E1842638
S113CA400BA78430890400BCCA0626EC3089FF5F3A
S113CA50BFCC2B8ECD03BFCC168ECADCBDCE81BD20
S113CA60CEB58D9EBDCEB58EC8408601A784BDD4FB
S113CA70062708A601BDD2007ECD678EC080BFCC3C
S113CA80148EC840BDD406270534307ED2D7BECC20
S113CA9014A780810D26E78EC840BDD1F48EC080D6
S113CAA0BFCC148ECD67BFCC437ED32E8ECAECBDD3
S113CAB0CE81BDCE2B8D1425F3B7CC0E8D0D25EC78
S113CAC0B7CC0F8D0625E5B7CC1039BDD175250B34
S113CAD0B6CC1C5D27031CFE391A013936383039AF
S113CAE020464C45582056332E3031044441544599
S111CAF020284D4D2C44442C5959293F200434
S113CC0008183A190004400000FF1B00010000004E
S113CC100000000000000000000000000000000010
S113CC200000000000000000000000BFFF00000141
S10ECC300000000000000000000000F5
S104CC496086
S113CC4E2B2B2B043F3F3F04574841543F04434191
S113CC5E4E2754205452414E53464552044E4F547F
S113CC6E20464F554E44044449534B204552524F8F
S113CC7E52202304445249564553204E4F542052B9
S113CC8E454144590447455400D20F4D4F4E00D3ED
S10DCC9E4B00271003E80064000AAD
S113CD007ECD577ECD677ECDB17ECD097ECD0C7EA6
S113CD10CD0F7ECD127ECEFB7ECF417ECE2B7ECE3E
S113CD20817ECFED7ECEB57ED00E7ECDEA7ED0362E
S113CD307ED1A27ED0EB7ED3497ECF867ECFD47EB9
S113CD40D27F7ED12F7ECFD07ED1757ED3297ECD6A
S113CD504E7ECE057ECE0510CEC07F7FCC11BDD4D5
S113CD60007FCC28BDD3FD10CEC07FBDDE188ECD94
S113CD7003BFCC168EC700AF9FD3E9BED3E7AF9FE6
S113CD80D3EB8ECCF8BFCC317FCC347FCC4C8D5AD6
S113CD90B6CC11B1CC0226057CCC1520147DCC2850
S113CDA010260597BDD40326B28ECC4EBDCE818D00
S113CDB07ABDD0D4810D27E58EC8407CCC0DBDD082
S113CDC03625168ECC938D3E2709BECC1227078DAF
S113CDD03526036E9801BDD22E8ECC568615B7CC5F
S113CDE020BDCE817FCC117ECD67BECD13BFCD10CB
S113CDF0BECD0DBFCD0A7FCC237FCC227FCC217F3B
S113CE00CC267FCC2439108EC844A6A0815F23028F
S113CE108020A18026086D8426F06DA4270C6D80E7
S113CE2026FC30026D8426DE1CFB398EC080BFCC0C
S113CE3014BDCEFBB1CC01271DB1CC00271F810D41
S113CE40270D810A2732811F23E78CC0FF27E2A721
S113CE5080810D26DC398ECC528D2620CE8CC0806C
S113CE6027F4301FB6CC07810826088620BDCF667C
S113CE70B6CC07BDCF6620B9860DBDCF4186202034
S113CE80C98D32A6848104276FBDCF41300120F3C0
S113CE90BDCD4E2765AD9FD3E5811312265C7FCCB3
S113CEA01AAD9FD3E58111122750810326F37FCC5D
S113CEB0116E9FCC167DCC2126278DD4B6CC0327AA
S113CEC020B1CC1A22187FCC1A7DCC0927028DCE32
S113CED03404F6CC0827058D085A26FB35047CCC8F
S113CEE01A860D8D5C860A8D583404F6CC05270607
S113CEF04F8D4E5A26FA35041CFE397DCC23261A52
S113CF007DCC2627108D1A7DCC2F27117DCC24278C
S113CF100C8D532008BDCD092003BDCD0C7FCC1A48
S113CF2039BFCC47BECC262006BFCC47BECC24BDDF
S113CF30D4062604BECC47397FCC24BDD27F7ECD17
S113CF40037DCC212620811F22057FCC2920177C3C
S113CF50CC293402B6CC04270BB1CC292406BDCE8F
S113CF60B57CCC29350234027DCC2226137DCC2419
S113CF7027048DB5200D7DCC262608BDCD0F2003BA
S113CF80BDCD123502397FCC4AF7CC1D8604B7CC0F
S113CF904DEC848ECCA08D0B30027ACC4D26F71F3D
S113CFA098203D7FCC4B10A3842507A3847CCC4BD5
S113CFB020F43402B6CC4B26107DCC4A260B7DCC13
S113CFC01D270B86208D2320057CCC4A8D123582AB
S113CFD08D023001A6848D04A68420044444444474
S113CFE0840F8B30813923028B077ECF418130251A
S113CFF014813923168141250C815A230E81612520
S113D00004817A23061A01B7CC11391CFE39341075
S113D010BECC14B6CC18B7CC19A680B7CC18810DE9
S113D0202710B1CC02270BBFCC1481202604A18485
S113D03027E78DB935908615A70186FFA7036F04EE
S113D0406F0CBDD0D48608B7CC4B8D34252E260F5B
S113D0508D2E25282609BCCC3F276C8D232368BE42
S113D060CC3F6D0427616D032A0F7DCC0D2705B6D7
S113D070CC0B2003B6CC0CA7037FCC0DBECC3F3920
S113D0808D8C254381392215BECC3F6D032A38840B
S113D09003A703BDD00E242F812E1CFE39F6CC4BE2
S113D0A02B253404C005F7CC4B3504B1CC492502FB
S113D0B08020A70430015ABDD00E2408812D2704F6
S113D0C0815F26065D26E41A01395D27CB6F0430A3
S113D0D0015A20F6BFCC3FBECC14A684812026047E
S113D0E0300120F6BFCC14BECC3F393430E60C26D8
S113D0F018108ED10B810B2210C6033D31A5C60337
S113D100A6A0A70C30015A26F735B042494E545810
S113D11054434D4442415353595342414B53435258
S113D1204441544241434449525052544F5554BDD2
S113D130D21EBDD00E25228D2625183404C60478AF
S113D140CC1C79CC1B5A26F73504BBCC1CB7CC1CA1
S113D1505C20DFBDD00E24FB39BECC1B1CFE398005
S113D160472A0F8B062A048B072A078B0A2B031CDA
S113D170FE391A0139BDD21EBDD00E25DC813922FB
S113D180D2840F34043402FCCC1B58495849584902
S113D190F3CC1BF3CC1BEBE08900FDCC1B35045C0A
S113D1A020D67FCC1D8D3D81022715811626F68D54
S113D1B033B7CC1E8D2EB7CC1F8601B7CC1D20E50E
S113D1C08D221F898D1E1E89F3CC1BFDCC3D8D1431
S113D1D01F894D27D08D0DBECC3DA780BFCC3D5AB5
S113D1E026F320C18EC840BDD4062711A6018108AC
S113D1F0260E32628604A784BDD406260D1CFE3991
S113D200B7CC20810426031A01398D737ECDE486C0
S113D210008D35250F8D077CCC4C8D8620F14F5F1A
S113D220FDCC1B39F6CC4C1027FBAE7ECD03860219
S113D2308D228DEABDD1A2F6CC1D27046E9FCC1E93
S113D2408ECC5C86817ECDDE34028EC840BDD03665
S113D2503502251A8EC840BDD0EB8EC8408601A782
S113D26084BDD1E4102500BB86FFA7883B39B6CC2A
S113D27011810D2707B1CC021026FB5D1A01393448
S113D28030A601B7CC202763BDCDEA10BECC2D2635
S113D2900881102758108ED3618EC8406D0227096B
S113D2A08604A784BDD406262E8EC838C60B8D6E80
S113D2B08EC840B6CC0BA7038601A784BDD406262E
S113D2C016B6CC204A47474C6F8820A7882186157C
S113D2D0A784BDD406271E8ECC75BDCE81BECC3F9F
S113D2E0B6CC20A7016F845FBDCF8635B08ECC82CB
S113D2F0BDCE8120F6BDCEB58EC840B6CC204A84C2
S113D30003C63F3DCB04E78822BDD40626C9BDCF62
S113D31041810D26F48604A784BDD40620CD343083
S113D3207ED1008ECC6B7ECDE13506FDCC4310FF63
S113D330CC457FCC207CCC287ECDB87FCC2810FE79
S113D340CC45F6CC206E9FCC433A397DCCFC2604E8
S113D3506E9FD3F38EC840861BA701BDD27F7ECDBE
S10FD360674552524F525300005359537A
S104CCC03936
S104CCD8391E
S104CCE43912
S10BCCF801000000000000002F
S113D37039396E9FF8046E9FF8006E9FF8086E9F0F
S109D380F80A6E9FF80696
S113D3E5D372D370E082E088D370D370D370D376D0
S113D3F5D371D37AD37ED3827ECA007ED4367ED4CB
S113D405597ED47B204449534B204F5045524154B7
S113D415494E472053595354454D20434F50595273
S113D4254947485420284329203139383020425966
S113D43520544543484E4943414C20535953544580
S111D4454D5320434F4E53554C54414E5453B7
S113D435FFBDDE158ED409C60A8D118E0005BFD435
S113D44513BFD4157FD41A8ED41BC61A6F805A26DF
S113D455FB7EC70CBDC709BED40927EB3088E4BFE2
S113D465D40B3420BDDAC3352024ECBED40B6F02B3
S113D475BDC70CC6FF397DCCFC2703BDC7093424C1
S113D485BFD40B6F01E6842622E602271AC10227C0
S113D49511BDD5B4BED40B25267DCCFC26235F3522
S113D4A52439BDD6CF20EDC6122014C1162304C6D7
S113D4B501200C5A588ED4CEAD95BED40B2402E768
S113D4C501BDC70C6D01352439D986D9D9DAF9DA04
S113D4D5C3D5E2D81DD838D876D641D69FD969DBCD
S113D4E5D6DB2CD699DA87D810D56FD590DB07DD36
S113D4F5BDDCFBDCE58D202605C6021A0139ED8469
S113D505AE846F846F01398D0E2705C60D1A013956
S113D515EC94ED841CFE39FCD40BC3001C8ED40999
S113D52510AE8426031CFB3910A384260139AE846E
S113D53520EEBED40B4F5F8D02C62FA78811300194
S113D5455A26F839BED40BC60BA604A78824300185
S113D5555A26F639BED40BC60BA6043402A6882473
S113D565A1E0260530015A26F039BED40BE6025453
S113D5752479E688237ED600BED40BE688226C88FF
S113D585223AA788405C261F1A0139BED40BE6024D
S113D595C403C1032655CA80E702E60FC580260ADF
S113D5A5E688233AA788401CFE39C60B1A0139A61A
S113D5B5883B2B3C27076A883B8620201D8D312517
S113D5C51B8118221527F68109260C8D23250DBEEE
S113D5D5D40BA7883B20D84D27E31CFE39BDDAB10F
S113D5E5250985012705A7847ED9A0C6121A013904
S113D5F5BED40BE68822270A6C88223AA688401CEA
S113D605FE398D0324EA39BED40BEC88406C88219D
S113D61526036C882010830000271CED881E340225
S113D6258604A7882235028D132410C5802704C6D5
S113D635102006C6092002C6081A01398D25BED454
S113D6450BBDDE0C25128D11BDDE0026031CFE3933
S113D65534048D17350424EE39BED40BEC881E3002
S113D6658840394FB7D411B7D41239C5102611C51E
S113D675802624F6D4115CC1072705F7D41120149C
S113D6857FD411F6D4125CC104270CF7D412BED48E
S113D6950BBDDE091CFE391A01398DC7BED40BBD7D
S113D6A5DE0C2520BED40B8DB0BDDE03260AB6D410
S113D6B5352737BDDE062732C540260B34048DAB2E
S113D6C5350424E039C6201A0139BED40BE6883B5B
S113D6D52B3D8120260F5CE7883BC17F260C200D5E
S113D6E58D0B24E6395D272720F61CFE393402C14B
S113D6F50126048620201086098D143502250F3451
S113D70502BED40BA6883B6F883B8D03350239BE18
S113D715D40BE602C1021026FED1E68822C10426F6
S113D7250834028D213502250FBDD57D240AC60492
S113D735BED40BE788221CFE39BED40B4F5FED889F
S113D74520ED88422027E688122622E688172744FA
S113D7556F88178D3F252A8DE025268DDC2522BE71
S113D765D40BC602E78817EC88117EDC828D0EBEC9
S113D775D40BED8840BDD69F241A7EDBC18D03EC06
S113D7858439BED40BE60386063D8ED41D3ABFD438
S113D7951B6D84398DE72605C6071A0139BED40BDE
S113D7A5ED88136D88122603ED88116C88162603FF
S113D7B56C88156D8817270BBDDC4325DDBED40B9E
S113D7C5EC8813BDD62025D2BED40BEC8840340694
S113D7D58DB03506ED84260A6F026F036F046F055D
S113D7E5200810AE04313F10AF044FBED40B6C8833
S113D7F52126036C88205FA7884030015A26F8BE8D
S113D805D40BEC8820ED88421CFE395F3404C60332
S113D815200EBED415BFD413F6D4133404F6D41491
S113D825BED40BE788413504E788407FD4185FE709
S113D835882239BED40BE68822261DBDD60C253098
S113D845BED40B7DD4182605DC44FDD4188610A758
S113D8558822EC881EED882FA68822A78831C61851
S113D8653414BDD5F53514A70430015A26F21CFE2F
S113D87539BED40BA68831A78822C6183414A60449
S113D885BDD714351430015A26F27ED69FBED40B6B
S113D895A603A78823B6D4177DD41A2631A703BEB9
S113D8A5D415BFD4138C0005270C8D222337BED481
S113D8B518BFD41320EFBED40BA68823A7032A0EC2
S113D8C5BDDDBD25368D07231CBDDDAD20F2BED4DF
S113D8D50B7FD41ABDD549BDD81DBDD8382407C181
S113D8E50827181A0139BED40BA604270C2A028D61
S113D8F50FBDD55926E41CFE398D051CFB1CFE39CC
S113D905A68833260CEC882FED8832A68831A788A3
S113D9153439BDD78726178D182515C60610BED4EC
S113D9250BBED41BA6A85D3121A7805A26F61CFE82
S113D93539BDD810BDD60C2508BED40BC610E78852
S113D9452239BDD7878DEA25F8C60610BED40BBE8D
S113D955D41BA680A7A85D31215A26F6BDD69F24DF
S113D965E07EDBC1BED40B8602A702EC882FED88CE
S113D9751EBDD6412508BDD87624057EDBC1C60A61
S113D98539BDD4FA253DBDD8922538263BBED40BE6
S113D9957DD41A2706A60F85202629BDDCC0252A95
S113D9A5EC8811ED8840BDDA76E688172713340430
S113D9B5BDD60C3504250C5A26F4BED40B5FE78876
S113D9C5221CFE39C6112002C6043404BDD50C350B
S113D9D5041A0139BED40B6D032A08BDDDBD240329
S113D9E5C61039BDD4FA25E2BDD537BDD91725DA18
S113D9F5BDD89225D52604C60320CFBDDCC025CAD3
S113DA05BED40BC60A6F0F30015A26F9BED40BECEF
S113DA1588322727ED882FA68834A78831FCCC0EB9
S113DA25ED8819B6CC10A7881BBDDDADBDD9692518
S113DA35998D3E8604A788221CFE39BED40B6F88B7
S113DA45176C8812EC882FBDD620250DBDD77225FD
S113DA5508BDD69F2406BDDBC17ED9CFBED40BEC51
S113DA65881EED88328610A78834BDD94725EA205B
S113DA758ABED40BA684A7026F846F883B4FA78800
S113DA8522398D28250E6F84441025FB7AC604E7B8
S113DA9588221CFE39BED40BA6028183260B86037D
S113DAA5A702BDD69F102501131CFE398DE7250D50
S113DAB5BED40BA602810323F0C6121A01398DECDC
S113DAC5253181022708BED40B6F027ED50CA688AA
S113DAD5122605BDDBA720198DC82517BED40B6DED
S113DAE588172705BDDC98250ABDD9692505BDD943
S113DAF54724D339BDD9862528BDD60C25238603CD
S113DB052018BDD986251ABED40BA60F85802612EA
S113DB15EC8813BDD62025098602BED40BA7021CAA
S113DB25FE39C60B1A01398D35BDD892252A27240D
S113DB35BED40BC60BA68824A70430015A26F68D3D
S113DB454D2515BED40BA60F858026D685602609DE
S113DB558D0C2055C6031A0139C60C1A0139BED4D9
S113DB650B860BB7D411A604E68835A78835E704D8
S113DB7530017AD41126EFBED40BA60C260CC603AD
S113DB85A6883DA70C30015A26F6BED40B398DCE96
S113DB95BDD89225072606BED40B1CFE39C6041A29
S113DBA50139BED40B86FFA704BDD969BED40B8643
S113DBB500A70239ED8840BDD69F2414C540260828
S113DBC5C580270AC6102006C60B2002C60A1A01FC
S113DBD539BDD917255E8DB8255ABED40BA60F8538
S113DBE580265285602652BDD787BED41BEC0226FB
S113DBF50FBED40BEC88112733BED41BED8420143F
S113DC05BED40BBDD620252CBED40BEC8811271C05
S113DC158DA22520BED40BEC8813BED41BED02BE09
S113DC25D40BEC8815BED41BE304ED04BDDBA7259A
S113DC3503BDD94739C60B2002C60C1A0139EC8835
S113DC451E5CE1883C2303C6014C10A38813260EF1
S113DC55A6883781FF27074CA788371CFE398D33E3
S113DC652530BED40BA6883A8B032616EC881E10E5
S113DC75A388112705C6171A0139EC8840ED8838A1
S113DC858604A7883AEC8813ED88358601A788377A
S113DC951CFE39EC8838BDD62025F7BED40B1F12DF
S113DCA5E6883A3AC603A6A8353121A7884030014B
S113DCB55A26F3BDD69F24DA7EDBC1BDD810BDD666
S113DCC50C2546BED40B4F5FED8820A68867A78830
S113DCD53C5F6F884030015A26F8BED40B1CFE39D0
S113DCE5BED40BA68817271DEC88208300012A03C0
S113DCF57EDD9AED8820BDDAB1250E4624076F84B2
S113DD05A688172605C6121A01397FD411EC881185
S113DD1510AE8820276ABDDD9F25EE4F5F6D022773
S113DD2574EB028900BFD40FBED40B10A388202442
S113DD352CBED40F30033402B6D4114CB7D41181A0
S113DD4554270881A83502274C20D23404BED40BAD
S113DD55EC88408D45253E3504350220C0A3882036
S113DD65BED40FA6023404A0E04A1F89A684EB01A1
S113DD75BED40B2505E1883C2306E0883C4C20F500
S113DD85BDD6202514BED40BEC884210A3882027C9
S113DD9514C6192002C6181A0139BDD6202508BE95
S113DDA5D40BC6443A1CFE39BED40BC60BA6882434
S113DDB5A70430015A26F639BED40BA6034C8104B8
S113DDC5240FA7032605BDDE0F2003BDDE1225E8BB
S109DDD539C6101A0139E1
S113DE007EDE317EDE907EDEB57EDEED7EDEF67E6B
S113DE10DF1B7EDF1B7EDE2F7EDE307EDE590000C0
S113DE2000000000000000000000000000000039B5
S113DE30391700258D3C347010BEDE2ACEF1005F08
S113DE40A6A0A7C05C26F98D41CEF1005FA6C0A7AD
S113DE50805C26F95F35F05F39B7DE2CF7DE2D8163
S113DE60302504803020F8B6DE2CF6DE2D1CFE1A98
S113DE704039B6DE2C8B10B7FFF9B6DE2D80018455
S113DE800F8B90B7DE2A7FDE2B398609B7FFF9396D
S113DE908DC73470CEF1005FA680A7C05C26F98DD3
S113DEA0D1CEF10010BEDE2A5FA6C0A7A05C26F981
S113DEB08DD85F35F017FFA134707FDE2E5F10BE62
S113DEC0DE2ACEF1008DABA6A0A7C05C26F98DBAE0
S113DED05FCEF100A680A1C027093404C618F7DE7E
S113DEE02E35045C26EEF6DE2E1CFE35F034124F81
S113DEF05F17FF6535923410A603810323014F8D0C
S113DF0012F6DE2CE784B7DE1E8D08A684B7DE2C5D
S112DF105F35908EDE20F6DE1E3A39A6035F39A8
